:020000040000FA
:040000000000C8280C
:08000800FD000308FE000A08D8
:10001000FF00830110100C10FC308F00FD308E00AB
:10002000AD0803191428AD03E623AE0B3B281E30A0
:10003000AE00B00B3B280530B000341E212834122E
:10004000222834164A26AF0B3B280230AF00C708DF
:10005000031D2C2835162E280130C702C808031DA1
:100060003328B51635280130C802B70803193B28D4
:10007000B70B3B28CB2110147F088A007E08830031
:10008000FD0E7D0E090082077E340C34B6349E349A
:10009000CC34DA34FA340E34FE34DE3400348034B6
:1000A000820700340134013402340334033404344D
:1000B000043405340634063407340834083409346B
:1000C0000934003482070C347234EC3480340C343C
:1000D000B6347E347E3480347E34CC3472340C3486
:1000E000F234A034A034B834A0340034BC34EE343C
:1000F000F034B034E9341034FE3480347E34DA34F1
:10010000FA3480349E340E34CC3480347E34CC3493
:1001100080347E34DA340A340034F234A034A1342A
:100120000034BC34EE34F034EE3403347E347034B6
:10013000023404347234B83470340C34E234EE34A3
:1001400008340C343834A034F23400340034003431
:100150000434A0342034A8340434EE34B8343834B1
:1001600004347C340234023404347C3410341034CB
:100170000434F034F23470340434A034F234CE3425
:100180000434EE340834A83404347234EE34703459
:10019000053084008001840A80300402031DCA28CF
:1001A0008001640083160313900170308F00831662
:1001B00003130F308100013085008601831603137D
:1001C000CE309F008312031381309F0083120313EC
:1001D000313090005A240F30BC00BB000230AE001A
:1001E000AF00B0003510D021C0308B008316031350
:1001F0000C148312031383161E3086008312D7213A
:1002000006190329FF2D83168601831200308D23E2
:10021000C2236400B9256F08D1007008D2003515DB
:100220001A2653241430AD0029216321B41E092954
:100230006400B31E2329341F23296F08D1007008DE
:10024000D20035151A2629213B08AD00532463211D
:100250001629B41A0800BD1831293D193129B410E6
:1002600008003D180800BD1837293D1D08006F081B
:10027000DB007008DC003E08DE003F08DF0081255F
:10028000611D54294008DE004108DF008125E11C82
:1002900054294308C800B512351E08003D195229DB
:1002A000B4100800B4140800B51E08004208C700C6
:1002B00035123D195D29B4145E29B4103A308D23EE
:1002C000FF30AD000800831603131E308600831232
:1002D0000313D721861979293418AC29D721861917
:1002E000A2293610341B7629341777293413DC21E0
:1002F000A229061987293418AC29D7210619A22961
:100300003611341B852935147729AA22A22986188B
:1003100095293418AC29D7218618A229B610341B88
:10032000932935107729AA22A229061A9E29341862
:10033000AC29D721061AA229B611A22934100F30F0
:10034000BC00BB008316031386018312031336140B
:10035000B6143615B6150800B41EC129341BB729CA
:10036000061AB7298619B729B701CB21C12905304B
:100370003C020319C029BB0BC129BC033C08BB00CC
:1003800034103614B6143615B615831603138601C9
:100390008312031308008724B412B30134133510F9
:1003A0004208C70035124308C800B512080064307F
:1003B000EB00EB0BD9290800831603138601831287
:1003C00003133414B416B101B2010F30B700341F57
:1003D000FA2933181A2AB3183A2A3319452AB319B5
:1003E000502A331A5E2AB31A682A331B732AB31BA6
:1003F000892A1A2A35180B2A33183A2AB318452A9B
:100400003319502AB3195E2A331A682AB31A732A89
:10041000331B892A1A2A3318892AB31B732A331BE0
:10042000682AB31A5E2A331A502AB319452A331997
:100430003A2A1A2AB3013314341B202A5930942A39
:100440003D1D292A0230A3007C30A4000230A50003
:100450000800BD1C322A1030A3006E30A4001030FA
:10046000A50008002030A300A830A400BC30A500DF
:100470003D140800B301B314341B402A4D30942AB4
:100480003E08D1003F08D2009A2AB3013315341B2D
:100490004B2A5130942A4008D1004108D2009A2AB0
:1004A000B301B315341B562A5D30942AD10142089A
:1004B000D200B11031113511C424A32AB30133166F
:1004C000341B642A4930942AD1014308D200592AA6
:1004D000B301B316341B6E2A6130942A6F08D10021
:1004E0007008D2009A2AB3013317341B792A453099
:1004F000942ABD1D822A7230A300F230A40070300D
:10050000A5000800BC30A300A030A400B830A500AE
:100510000800B301B317341B8F2A5530942A1830C2
:100520008D2355308D2308003518982A8D23080017
:10053000A72308003515C424BD19A12AB11431110F
:10054000A32AB11031155308A5005408A40055087A
:10055000A3000800831603138601831203133414C7
:100560000F30B7003318C12AB318232B33194C2B83
:10057000B319722B331A082BB31AE52A331BDF2A5F
:1005800008003619D02A3D1CC82A3D10BD14202A67
:10059000BD1CCD2ABD103D15202A3D113D14202A39
:1005A000B618202A3D1CD72A3D103D15202A3D1D96
:1005B000DC2A3D11BD14202ABD103D14202ABD1D8A
:1005C000E32ABD11E42ABD15792A3619F72A7F30AE
:1005D000DB00FF30DC004408DE004508DF00812539
:1005E000E11CF72A0530C5070318C40A072BB61803
:1005F000072BDB010130DC004408DE004508DF008A
:100600008125611D072B0530C502031CC4036E2A1A
:10061000B618162BDB01F030DC00DE014308DF00EA
:100620008125E11C162B0130C307222B3619222B02
:10063000DB01DC01DE014308DF008125611D222B87
:100640000130C302642AB618352B0330DB00E730D3
:10065000DC003E08DE003F08DF008125E11C352B71
:100660000130BF070318BE0A4B2B36194B2B40082D
:10067000DB004108DC000A30DC070318DB0A3E0817
:10068000DE003F08DF008125611D4B2B0130BF02DA
:10069000031CBE034B2B402AB618622B3E08DB001E
:1006A0003F08DC000A30DC02031CDB034008DE00EC
:1006B0004108DF008125E11C622B0130C1070318CE
:1006C000C00A712B3619712BDB01DC014008DE00FA
:1006D0004108DF008125611D712B0130C102031C1F
:1006E000C0034B2AB618802BDB01F030DC00DE01A2
:1006F0004208DF008125E11C802B0130C2078C2BD2
:1007000036198C2BDB01DC01DE014208DF0081257C
:10071000611D8C2B0130C202562AAA00B101C223EE
:100720002A08EA006220E900EA0AE90B982B08008F
:1007300064002408A3002508A4006A086220A5001C
:100740006400AD08031DA02B4130AD00942BAA001E
:10075000B101D4232A08EA006220E900EA07EA038B
:10076000E90BB32B080064002408A5002308A400AB
:100770006A086220A3006400AD08031DBB2B413052
:10078000AD00AF2B0430EA00EA0BC72B0800640071
:100790002408A3002508A400A5016400AD08031DDA
:1007A000CD2B4130AD00C42B0430EA00EA0BD92B2D
:1007B000080064002408A5002308A400A301640025
:1007C000AD08031DDF2B4130AD00D62B32182314AA
:1007D000B1182414311925142C1CFF2B2308A00058
:1007E000311FF72B341EF72B0130A005F72BB11D5D
:1007F000FB2B341E20102324AC01AC140800AC1CCD
:10080000122C2408A000B11F0A2C341E0A2C01301F
:10081000A0050A2C311E0E2C341E20102324AC01FE
:100820002C1508002508A000311C1B2C341E1B2C85
:100830000130A0051B2CB11E1F2C341E20102324B8
:10084000AC012C1408000608A1000508A200003025
:10085000A2058630A2040130A1050030A1042208BF
:1008600085002108860020182217A018A11420193D
:100870002115A019A115201A2116A01AA116201BB6
:100880002117A01BA1172C18A210AC1822112C198B
:10089000A213B4184D2C21104E2C211422088500CF
:1008A0002108860008006400AD08031D532C3C306D
:1008B000AD0008000A30BA003D308400B80166245B
:1008C0008000840AB80ABA0B5F2C08007824390823
:1008D000A900B80A782439082902031D712C3908A7
:1008E0000800031C752C3908762C290834150800DB
:1008F0003808831203178D00831603178C130C140A
:10090000831203170C0883120313B90008000B08A5
:10091000AB008B130A30BA003D308400B8010008E8
:100920009824840AB80ABA0B8F2C2B088B00080075
:10093000B900AA00A024B80A2A08B900A024080017
:10094000831603178C18A22C8C130C158312031317
:100950003808831203178D0083120313390883129A
:1009600003178C008316031755308D00AA308D00B5
:100970008C14831203130800831603178C18BE2CE3
:100980000C118312031308005008EC005108ED000D
:100990005208EE00B411B518D12CD001D11FDF2CB4
:1009A000D42CD01FDF2CD009B415D209D1090130C5
:1009B000D207031CDF2CD107031CDF2CD00AB51093
:1009C00003101830CA00CC01CD01CE01CF01D20DE9
:1009D000D10DD00DCF0DCE0DCD0DCC0DCA0B692D87
:1009E0004C080F39D9004D0E0F39D8004D080F397A
:1009F000D7004E0E0F39D6004E080F39D5004F0ED6
:100A00000F39D4004F080F39D3000A30D908031D1D
:100A1000262DD900D808031D262DD800D708031D80
:100A2000262DD700D608031D262DD600D508031D78
:100A3000262DB51D1D2DB511262DD500D408031D5D
:100A4000262D351D252D3511262DD400B41D4D2DF7
:100A50000A305402031D2F2D0B30D4004D2D0A30C7
:100A60005502031D362D0B30D5004D2D0A30560290
:100A7000031D3D2D0B30D6004D2D0A305702031DAE
:100A8000442D0B30D7004D2D0A305802031D4B2D3D
:100A90000B30D8004D2D0B30D90059084320D90018
:100AA00058084320D80057084320D7005608432051
:100AB000D60055084320D50054084320D4005308DD
:100AC0004320D3006C08D0006D08D1006E08D2001E
:100AD00000344F30840076254E30840076254D302A
:100AE000840076254C3084007625E72C03300007FF
:100AF000CB00CB19800030300007CB00CB1B80002F
:100B00000034E101E001DB1B6014DE1BE014E008AF
:100B10000319982D01306002031D912D6115611696
:100B2000080002306002031D982DE114E115080051
:100B30005B085E02031D9D2DA72D5B085E02031856
:100B4000A42DE114E11508006115611608005C0888
:100B50005F02031DAF2D61146116E11508005C08EA
:100B60005F020318B62DE114E11508006115611646
:100B700008003F08DC003E08DB00E730DF00033000
:100B8000DE008125E118FF2DDF01DE0181256119DD
:100B9000FF2D4108DC004008DB00E730DF000330B8
:100BA000DE008125E118FF2DDF01DE0181256119BD
:100BB000FF2D4208DC00DB01F030DF00DE01812583
:100BC000E118FF2DDF01DE0181256119FF2D4308AA
:100BD000DC00DB01F030DF00DE018125E118FF2DB4
:100BE000DF01DE0181256119FF2D4508DC00440885
:100BF000DB00DF01DE0181256119FF2D080083166E
:100C00000313860183120313BD01BE01F030BF0040
:100C1000C0010A30C1000A30C2000A30C30080306F
:100C2000C5002530C4008724B410B101B2012830BA
:100C30008D23142EC4245108DB005208DC0003303D
:100C4000DE00E730DF008125E11C2A2E32308D23C3
:100C5000C2230800BD193B2EB41C302E3116312E94
:100C60003112B1123111B1145308A5005408A40077
:100C70005508A3000800B41C3F2EB116402EB11237
:100C800031123115B1105308A5005408A4005508BD
:100C9000A3000800F2080319512E0230F202031DCE
:100CA000532E0830F2001F151F19542E7230720790
:100CB000840083161E08831280001E0884038000AF
:100CC0007A3084000008FC0084030008FB00033035
:100CD000F10084030008FC070318FB0A84030008E2
:100CE000FB07F10B692E0310FB0CFC0C0310FB0C33
:100CF000FC0CDA017B08DB007C08DC00DD0127301E
:100D0000DE001030DF0095265F08DA006308DB00A4
:100D10006408DC00DD014408DE004508DF00CE2663
:100D20005B08EF005C08F00008005B085E06E80066
:100D3000DE1F9F2EDF09DF0A0319DE03DE09DB1F3A
:100D4000A62EDC09DC0A0319DB03DB091030CB001B
:100D50005E08E6005F08E700DE01DF01BF26CB0B7F
:100D6000AE2EE81F0034E409E309DF09DE09E40AD6
:100D70000319E30A0319DF0A0319DE0A0034E60C3B
:100D8000E70C031CC92E5C08DF070318DE0A5B08AA
:100D9000DE07DE0CDF0CE30CE40C0800E201E301EB
:100DA000E401CB015A0DE40D5F08E4025E08031C68
:100DB0005E0FE3025D08031C5D0FE2020030031CBE
:100DC0000130CB02DA0D0730E0005A0DE40DE30DDF
:100DD000E20DCB0D5F085A1CFB2EE4025E08031CDB
:100DE0005E0FE3025D08031C5D0FE2020030031C8E
:100DF0000130CB02082FE4075E0803185E0FE307FB
:100E00005D0803185D0FE207003003180130CB07BF
:100E1000DA0DE00BE52E5B0DE40DE30DE20DCB0DDD
:100E20005F085A1C212FE4025E08031C5E0FE302D8
:100E30005D08031C5D0FE2020030031C0130CB0291
:100E40002E2FE4075E0803185E0FE3075D08031802
:100E50005D0FE207003003180130CB07DB0D0730D0
:100E6000E0005B0DE40DE30DE20DCB0D5F085B1CB4
:100E7000472FE4025E08031C5E0FE3025D08031CBB
:100E80005D0FE2020030031C0130CB02542FE40757
:100E90005E0803185E0FE3075D0803185D0FE207A5
:100EA000003003180130CB07DB0DE00B312F5C0D58
:100EB000E40DE30DE20DCB0D5F085B1C6D2FE4022A
:100EC0005E08031C5E0FE3025D08031C5D0FE20277
:100ED0000030031C0130CB027A2FE4075E080318B0
:100EE0005E0FE3075D0803185D0FE207003003188B
:100EF0000130CB07DC0D0730E0005C0DE40DE30DA5
:100F0000E20DCB0D5F085C1C932FE4025E08031C0E
:100F10005E0FE3025D08031C5D0FE2020030031C5C
:100F20000130CB02A02FE4075E0803185E0FE30731
:100F30005D0803185D0FE207003003180130CB078E
:100F4000DC0DE00B7D2F5C18AF2F5F08E4075E0817
:100F500003185E0FE3075D0803185D0FE207003416
:100F60000028002800280028002800280028002841
:100F70000028002800280028002800280028002831
:100F80000028002800280028002800280028002821
:100F90000028002800280028002800280028002811
:100FA0000028002800280028002800280028002801
:100FB00000280028002800280028002800280028F1
:100FC00000280028002800280028002800280028E1
:100FD00000280028002800280028002800280028D1
:100FE00000280028002800280028002800280028C1
:100FF00000280028002800280028002800280028B1
:02400E00740834
:104200000000000000000000F000F00000000000CE
:104210000A000A000A000A000A000A002500250018
:08422000800080000000000096
:00000001FF
